:100000000C9434000C9458030C944C020C94510042
:100010000C9451000C94A8010C9451000C945100C4
:100020000C9451000C9451000C9451000C9451000C
:100030000C9451000C9451000C9451000C945100FC
:100040000C9451000C9451000C9453000C945100EA
:100050000C9451000C9451000C9451000C945100DC
:100060000C9451000C94510011241FBECFEFD8E026
:10007000DEBFCDBF13E0A0E0B1E0E0E2FBE002C0F4
:1000800005900D92A030B107D9F714E0A0E0B3E0DD
:1000900001C01D92A732B107E1F70E94DB030C9467
:1000A0008E050C9400001F920F920FB60F92112430
:1000B0008F939F93EF93FF9380912404813049F5B0
:1000C00080910203E82FF0E09091C600EC56FC4FBF
:1000D00090838F5F8093020380910203843091F5B7
:1000E0001092020380919403809392038091950370
:1000F00080931C0480919603809311038091970351
:1001000080939803809192038C34E1F4109224043C
:1001100019C0809124048823A9F480910203E82F58
:10012000F0E09091C600E756FC4F90838F5F80937C
:10013000020380910203803829F41092020381E0C7
:1001400080932404FF91EF919F918F910F900FBEA8
:100150000F901F90189585B5846085BD85B58D7FFE
:1001600085BD85B58E7F85BD569A84B5836084BD77
:1001700084B5806884BD80EE87BD089589E1809351
:10018000C4001092C50088E98093C1001092020358
:1001900008959091C00095FFFCCF8093C60008950C
:1001A0008091C00087FFFCCF8091C60008955298CF
:1001B0005A9AE9E6F0E0808182608083E09AE89ACA
:1001C0000895E9E6F0E0808188608083E8980895EA
:1001D000F8940E94E1007894E19AE99A08951092C7
:1001E0000003DA9AEDE6F0E080818061808380810F
:1001F0008F7D808380818F778083DA9A0895F89449
:100200000E94EF007894DA9AE8E6F0E0808184605A
:100210008083089581E080930003DA9AEDE6F0E0B0
:1002200080818062808380818F7E808380818F77D0
:100230008083DA9A0895F8940E940A017894DA9AF1
:10024000E8E6F0E0808184608083089582E0809316
:100250000003DA9AEDE6F0E0808180688083808197
:100260008F7E808380818F7D8083DA9A0895F894D1
:100270000E9426017894DA9AE8E6F0E080818460B2
:10028000808308953898409AD89AEDE6F0E080810E
:1002900081608083D89A08950E94E80083ED90E3FE
:1002A0000197F1F700C000000E94FF0083ED90E38A
:1002B0000197F1F700C000000E941B0183ED90E35D
:1002C0000197F1F700C000000E94370183ED90E331
:1002D0000197F1F700C000000895883018F41092DB
:1002E000010332C0982F98509E3010F481E02AC04C
:1002F000982F96519E3010F482E024C0982F94528B
:100300009D3010F483E01EC0982F91539C3010F460
:1003100084E018C0982F9D539E3010F485E012C0E1
:10032000982F9B549D3010F486E00CC0982F985560
:100330009D3010F487E006C085568E3010F488E0BA
:1003400001C089E0809301038091010390E008954A
:100350001F920F920FB60F9211242F933F934F933A
:100360005F936F937F938F939F93AF93BF93EF931D
:10037000FF93809168008B7F8093680080910003D9
:10038000882331F589B190E08071907034E09595C3
:1003900087953A95E1F78093250480912504813073
:1003A00029F480916800846080936800809125041E
:1003B000882371F4809168008B7F8093680086B5F4
:1003C00080932604809126040E946D0180931B0473
:1003D00080910003813031F589B190E08072907096
:1003E00025E0959587952A95E1F7809325048091DE
:1003F0002504813029F4809168008460809368002E
:1004000080912504882371F4809168008B7F80930C
:10041000680086B580939303809193030E946D01D9
:100420008093210480910003823029F589B1881FCF
:100430008827881F8093250480912504813029F422
:1004400080916800846080936800809125048823EF
:1004500091F4809168008B7F8093680086B58093CB
:100460000C0380910C030E946D0180930403809122
:1004700004030E94C900FF91EF91BF91AF919F913A
:100480008F917F916F915F914F913F912F910F903D
:100490000FBE0F901F9018951F920F920FB60F92DC
:1004A00011242F933F934F935F936F937F938F9379
:1004B0009F93AF93BF93EF93FF93E99886B5809393
:1004C0002304809123040E946D0180930B03FF910C
:1004D000EF91BF91AF919F918F917F916F915F91BC
:1004E0004F913F912F910F900FBE0F901F90189535
:1004F000309198032091110380911C0490E0A0E0BA
:10050000B0E0DC0199278827830F911DA11DB11D43
:10051000522F40E060E070E0840F951FA61FB71FC8
:1005200080931D0490931E04A0931F04B093200495
:100530000895CF92DF92EF92FF9230910B0380915A
:100540001B04909121046091040320910503482F1E
:1005500050E06A01CC0CDD1CE3E0440F551FEA9526
:10056000E1F7C40ED51EEE24D7FCE094FE2C84E601
:10057000989FC0011124AA2797FDA095BA2FC80EF5
:10058000D91EEA1EFB1EC30ED11CE11CF11C70E03B
:1005900048EE53E0649FC001659F900D749F900DDD
:1005A0001124AA2797FDA095BA2FC80ED91EEA1EBE
:1005B000FB1E30E040E050E0C701B6010E944D054F
:1005C000DC01CB0180930D0390930E03A0930F03E6
:1005D000B0931003813523EC920720E0A20720E0BE
:1005E000B20760F080E593ECA0E0B0E080930D03EB
:1005F00090930E03A0930F03B093100360910D032B
:1006000070910E0380910F03909110032FE931E157
:1006100040E050E00E944D0524E630E040E050E02C
:100620000E946C0520931D0430931E0440931F0408
:1006300050932004FF90EF90DF90CF900895809129
:100640001D0490911E04A0911F04B09120044091BC
:100650000703509108036091090370910A03840F06
:10066000951FA61FB71F8093070390930803A093BD
:100670000903B0930A03EA2FE695E0931904F0E02A
:10068000EE5EFC4F808185B9809192038234B9F689
:10069000089540E0242F30E0FC01E20FF31F508169
:1006A0002E5E3C4FF90150834F5F403899F7089513
:1006B0001F920F920FB60F9211242F933F934F93D7
:1006C0005F936F937F938F939F93AF93BF93EF93BA
:1006D000FF93E8980E944C0182E4809392038FE993
:1006E00096E8A1E081509040A040E1F700C00000F2
:1006F000E89A86B1817080931A0486B190E0827086
:100700009070959587958093030380911A048823B0
:1007100011F481E001C08AE0809305031092070381
:10072000109208031092090310920A030E94990282
:1007300080910303882319F480E892E002C080E0EE
:1007400092E00E94490381E4809392030E941F0378
:10075000FF91EF91BF91AF919F918F917F916F9199
:100760005F914F913F912F910F900FBE0F901F906F
:1007700018958091070390910803A0910903B09107
:100780000A0388599047AF4FBF4F80930703909358
:100790000803A0930903B0930A03EA2FE695E093B8
:1007A0001904F0E0E058FD4F808185B980919203F3
:1007B0008234F9F608958FEF84B93898409A3998C1
:1007C000419A0E94BE00F8940E94D70078940E943B
:1007D000AB0082E48093920381E080932404CAE218
:1007E00087EA91E60197F1F700C00000809192033B
:1007F0008335A1F5109207031092080310920903A4
:1008000010920A030E94780284E40E94C90084E4E2
:100810000E94C90083E50E94C9008FE50E94C900BB
:1008200083E50E94C90089E60E94C9008EE60E9405
:10083000C9008FE50E94C90083E50E94C90085E6D2
:100840000E94C90084E70E94C9008DE00E94C9008F
:100850008AE00E94C90080E892E0F1C08091920392
:100860008435A1F510920703109208031092090332
:1008700010920A030E94780284E40E94C90084E472
:100880000E94C90083E50E94C9008FE50E94C9004B
:1008900084E50E94C90082E70E94C90089E60E949F
:1008A000C9008FE50E94C90083E50E94C90085E662
:1008B0000E94C90084E70E94C9008DE00E94C9001F
:1008C0008AE00E94C90080E092E0B9C08091920362
:1008D0008535E9F510920703109208031092090379
:1008E00010920A030E94780284E40E94C90084E402
:1008F0000E94C90083E50E94C9008FE50E94C900DB
:1009000082E50E94C90081E60E94C9008DE60E942E
:10091000C90080E70E94C90085E50E94C90080E700
:100920000E94C9008FE50E94C90083E50E94C900AA
:1009300085E60E94C90084E70E94C9008DE00E94FC
:10094000C9008AE00E94C90080E891E078C08091E7
:1009500092038434E9F51092070310920803109271
:10096000090310920A030E94780284E40E94C900DD
:1009700084E40E94C90083E50E94C9008FE50E94BB
:10098000C90082E50E94C90081E60E94C9008DE687
:100990000E94C90080E70E94C90084E40E94C90047
:1009A0008EE60E94C9008FE50E94C90083E50E947F
:1009B000C90085E60E94C90084E70E94C9008DE055
:1009C0000E94C9008AE00E94C90080E091E037C01F
:1009D000809192038134C1F51092070310920803AD
:1009E0001092090310920A030E94780284E40E9484
:1009F000C90084E40E94C90083E50E94C9008FE514
:100A00000E94C90081E40E94C90082E70E94C900D7
:100A100082E60E94C9008FE50E94C90083E50E941A
:100A2000C90085E60E94C90084E70E94C9008DE0E4
:100A30000E94C9008AE00E94C90089E993E00E94EF
:100A400049030E941F03CCCE80919203893409F0A0
:100A5000C7CE81E40E94C9008AE60E94C9008FE5E2
:100A60000E94C90083E50E94C90089E60E94C9006E
:100A700087E60E94C90087E40E94C90085E60E94BB
:100A8000C9008EE60E94C9008DE00E94C9008AE07C
:100A90000E94C900C0939203A3CE629FD001739FAE
:100AA000F001829FE00DF11D649FE00DF11D929F0A
:100AB000F00D839FF00D749FF00D659FF00D992749
:100AC000729FB00DE11DF91F639FB00DE11DF91F6D
:100AD000BD01CF0111240895A1E21A2EAA1BBB1B50
:100AE000FD010DC0AA1FBB1FEE1FFF1FA217B307FA
:100AF000E407F50720F0A21BB30BE40BF50B661F10
:100B0000771F881F991F1A9469F7609570958095D3
:100B100090959B01AC01BD01CF010895F894FFCFE2
:100B20003F3E3E3D3D3C3C3B3B3A3A393938383715
:100B30003736363535343433333232313130302F85
:100B40002F2E2E2D2D2C2C2B2B2A2A2929282827F5
:100B50002726262525242423232222212120201F65
:100B60001F1E1E1D1D1C1C1B1B1A1A1919181817D5
:100B70001716161515141413131212111110100F45
:100B80000F0E0E0D0D0C0C0B0B0A0A0909080807B5
:100B90000706060505040403030202010100000024
:100BA0000000000101020203030404050506060714
:100BB00007080809090A0A0B0B0C0C0D0D0E0E0F85
:100BC0000F101011111212131314141515161617F5
:100BD00017181819191A1A1B1B1C1C1D1D1E1E1F65
:100BE0001F202021212222232324242525262627D5
:100BF00027282829292A2A2B2B2C2C2D2D2E2E2F45
:100C00002F303031313232333334343535363637B4
:100C100037383839393A3A3B3B3C3C3D3D3E3E3F24
:100C20001F202122232425262728292A2B2C2D2E5C
:100C30002F303132333435363738393A3B3C3D3E4C
:100C40003F3E3D3C3B3A393837363534333231302C
:100C50002F2E2D2C2B2A292827262524232221201C
:100C60001F1E1D1C1B1A191817161514131211100C
:100C70000F0E0D0C0B0A09080706050403020100FC
:100C800000000102030405060708090A0B0C0D0EFB
:100C90000F101112131415161718191A1B1C1D1EEC
:100CA0001F2122242527282A2B2D2E30313233359F
:100CB000363738393A3A3B3C3D3D3E3E3E3F3F3F7A
:100CC0003F3F3F3F3E3E3E3D3D3C3B3A3A39383761
:100CD0003635333231302E2D2B2A28272524222158
:100CE0001F1E1C1B191816151312100F0E0C0B0AC1
:100CF00009080706050403030201010000000000C3
:100D000000000000000001010203030405060708BB
:100D1000090A0B0C0E0F101213151618191B1C1EA6
:00000001FF
